:100000007581500200067D007F007B64120110DBC9
:10001000FB7B6412002480F435673369316A3668EB
:100020003273346E30931730922230912C309036E8
:10003000D297D296D295D2947D0012009422C29784
:10004000C296C295C2947F0012007322D297C296C4
:10005000C295C2947D007F0022D297D296C295C2EB
:10006000947D007F0022D297D296D295C2947D00D3
:100070007F0022BD000302007EBD06137D009001BB
:10008000201200B51201199002301200B50D221293
:1000900000EA0D22BF000302009FBF0B137F0090F8
:1000A00001201200B51201199003811200B50F2230
:1000B0001200EF0F22E493B4FF03D2B2227908A218
:1000C000E792B21200F223D9F6A380E97EC8C2B249
:1000D000120100D2B2120100DEF4227EFAC2B21284
:1000E00000F9D2B21200F9DEF42211CC11CC2211A7
:1000F000CC22750830D508FD2275084BD508FD22A5
:10010000750860D508FD2275090A11F2D509FB2290
:10011000750A0A3107D50AFB227C0A3110DCFC2261
:10012000AAB2AAAD554A56CA7A253751BA2A93B10E
:100130005D8AA2BA2ED1A49E86F0B427B0DD1A44FF
:10014000F86F25913E1BD1644F86F45887B1BA2CC5
:1001500089D8B74A91763746917659D2A45B2DA9B2
:1001600048BB2CD9522DAAD5522DAAD54A4DAAD575
:100170005295AAD554956AD654956AD655256AD60D
:1001800095256AD69525AB5A9526AD5A952AB56A16
:1001900094AAB56A549AB5AA54AB56A952AB56A5BF
:1001A0004AAB56A54AB56A954AB56A952AB56A54C6
:1001B000AAB555554AAB55552AAAB5554AAAAD55C3
:1001C00052AAAB5555555555555555555555555537
:1001D00055555555555555555555555555555555CF
:1001E00055555555555555555555555555555555BF
:1001F00055552D555555555555555552B5652A6D7D
:10020000A949AB6A492EDA912BB6A215ED94837BEE
:100210006508DDB290AF6CA11BEB4225ED94237D08
:100220006904FD56116ED5411FB5502DECB40AFF7F
:100230002529DA5AAB2AA578BA56564CBC5E569692
:100240009574AE969A9574B655552AE4EAAAAA56BC
:10025000CAD4D5525E2D95554AE8DA9AAA53C5B24A
:10026000AAA93C574ACA8BC574AD28BC5745D24B86
:10027000C4F45A92791DA3648F91DC3690F61BC4A6
:10028000D48ED29D4AA9AAAAAAAAAAAAAAAAAAAA06
:10029000AAAAAAAAA55AAAAAA955AA56AA52DA95FA
:1002A0006AA4B5A556A9556AAAAAA5555555552BB0
:1002B0005555554AB5555554AAD55554AAB5555511
:1002C00055555555555555555555555555555555DE
:1002D00055555555555555555555555555555555CE
:1002E00055555555555555555555555555555555BE
:1002F00055555555555555552D5555552AD6955540
:1003000049AD9555496DA2D690BEA17A913D917A9D
:10031000895D917A4A5752B68AA754AE92A5D4AD58
:10032000A2A5D92BA4A96D2B64A9762B692A765294
:10033000F2527692DA925D92BA925DA4BA9257A87E
:10034000AEA897AA2DA916EC8D6A276A95A52B5AF7
:10035000AAA92B6AAAA8AB6AAAA4AD6AAAA4AD6A84
:10036000AAA4AD6AAAA4AB5AAAA4AB5AAA52AB5A81
:10037000AA94AB5AAA94AB5AAAA4AB5AAAA4AB5A51
:10038000FFAAA9A69A71AAAAAAAAAAAAAAAAAAAAC6
:10039000AAAAB555555556AAAAAAAAAAAB55AAAA59
:1003A000A5554AA94A54AA54AA9552AAAAAAAAA5E6
:1003B00055555555556AD6B56AAAA9529564D2CAFB
:1003C000AAA9569D2D2D2CA8F0F4B4B4A94F0F5214
:1003D000D34B24F0EA6CB4B13E1DA74E4D2787A93C
:1003E000D352A5E1E65AB468BC3B1D568C4F0F476B
:1003F000556313C3B174B4A4F0EC5B4D293E178A66
:10040000E34A4F85E2B95293C4F49D2A92785D8BFA
:10041000A8A93C8ED1B492BC8BD26D225E86EA56DE
:10042000525ACAAAAAAA555AAAAAA9555AAAAAA504
:10043000556AAAAA9555AAAAAA5556AAAAA9555A6A
:10044000AAAA9555AAAAA95556AAAAA5556AAAAABA
:10045000555AAAAA9555AAAAA9555AAAAA9556AA1A
:10046000AAA5556AAAA9555AAAAA5556AAAAA5552F
:10047000AAAAA5555AAAA9555AAAAA5556B2CA4D0A
:10048000AD95524DB55551376AAA89BB555513B62E
:100490009A9436DA55215DAAA90ADD55511B755586
:1004A000215BAAAA4376AAA90DDAAAA2376AAA846E
:1004B000BDAAA90AF6AAA44BDAAA90AF6AAA42BDBD
:1004C000AAA90AEEAAA42BBAAA90AEEAAA42B76ACF
:1004D000A912DEAAA506EEAA541BBAAA90AEECAAEF
:1004E0008877AAA511BB695483BD555215DD5549BE
:1004F0001BB65548ADDAAAFFFF35673369316A3656
:06050000683273346EFF47
:00000001FF
